:020000040000FA
:10000000F86A7D0EF76EC00EF66EA68EA69CA684CC
:10001000A688F29E550EA76EAA0EA76EA6820000B5
:10002000F28E010EF56E0D00EF0EF56E0D00300E26
:10003000F56E0D00F00EF56EF56A0D000D000D0069
:100040000C00A68EA69CA684A698F29E550EA76EBE
:10005000AA0EA76EA6820000F28EA6948E0EC16E26
:10006000E10E926E100E806E8082FFD701EF30F0AD
:10600000FFD7E0CF0AF50501F2AE03D0F29E128F62
:1060100001D0129FE8CF00F5D8CF01F5EACF02F505
:10602000E9CF03F5E2CF04F5E1CF05F5DACF06F5C8
:10603000D9CF07F5FBCF08F5FACF09F5F8CF0BF567
:10604000F7CF0CF5F6CF0DF5D5AE03D0D59E128166
:1060500001D01291CDA003D0CD90128301D0129324
:10606000CAA403D0CA94128501D01295B1A003D05E
:10607000B190128701D01297D49CBDEC30F059B585
:1060800001D0396BC4EC30F05851130B130A20E0E7
:1060900059B506D0596BC9EC36F06CEC35F001D02F
:1060A0005995126B0E6B0F6B106B116B58B310D0B0
:1060B000700EF76E980EF66E0BEC31F0700EF76EF8
:1060C000BC0EF66E0BEC31F016EC31F09DEC31F0BD
:1060D00058AB24D0D4AA05D010C50EF511C50FF5C4
:1060E0001DD058AF12D080EC31F039B901D03983CE
:1060F000FECF10F5FDCF11F5710EF76E100EF66E96
:106100000BEC31F09DEC31F009D0D488B8500E6F13
:10611000B7500F6FD498D8900F370E37FECF10F5C9
:10612000FDCF11F558AB1AD0589B58AF0AD0D4BA4E
:1061300008D09EAA06D0710EF76E100EF66E0BEC0C
:1061400031F058AD09D0589DD6EC36F0710EF76E8F
:10615000100EF66E0BEC31F01DEC37F0710EF76E91
:10616000100EF66E0BEC31F0598147EC32F059917C
:10617000FCEC32F09DEC31F0F1D71F0EAF6EAC8429
:10618000AC8AAB88AB8E1200FCAC07D0FC9C740EC2
:10619000F76E560EF66E0BEC31F0FCAE07D0FC9E9F
:1061A000740EF76E440EF66E0BEC31F0D0501F0BF0
:1061B0001F0A0DE158AB0AD058AF07D0D4BA05D0AA
:1061C000A9EC32F09EBA01D0D09201D0D092D0B2D8
:1061D00006D0DD0E586F596BD082D08001D0588325
:1061E000D0B009D05891D080740EF76E280EF66E9C
:1061F0000BEC31F001D05881D0B80BD05899D08831
:1062000059B506D0730EF76EDE0EF66E0BEC31F05C
:1062100001D0588912000800F55004D80B00F55041
:10622000FCE112009EA8FED7AD6E120080EC31F0AA
:1062300039B947D09EAA03D0AE509EBAFDD7020E00
:10624000136F1353D8B431D0730EF76E060EF66E7B
:106250000BEC31F0730EF76E2A0EF66E0BEC31F08C
:106260005B0E12EC31F0200E12EC31F0132FFBD745
:106270005D0E12EC31F0030E136F080E12EC31F0CC
:10628000132FFBD7020E136FABA202D0AB98AB88D3
:106290009EBA15D0640E146FA9EC32F01407FCE11D
:1062A000230E12EC31F0132FEFD7B9EC32F0710E50
:1062B000F76E100EF66E0BEC31F0398102D0B9ECAE
:1062C00032F012003989000EF76E000EF66E030EE2
:1062D000156F0900F55207E00900F550EF0801E1DC
:1062E00039990DD00AD00900F550EF0803E139992A
:1062F00006D003D0F55001E002D01507EAE1120004
:106300003989F76AF66A600E616F000E626F0900E4
:10631000F550FF0A01E009D0620701E2610762530C
:1063200003E1615301E101D0F2D7615304E162530B
:1063300001E0399901D03999120039AD09D0C9EC81
:1063400033F0710EF76EEE0EF66E0BEC31F01DD0E1
:1063500039AF09D0C9EC33F0720EF76E0C0EF66E41
:106360000BEC31F012D039A907D0720EF76E340E53
:10637000F66E0BEC31F009D039A303D0C7EC31F045
:1063800004D039A102D003EC32F0396B12000600C0
:1063900006005851130B130A07E0FC2A000EFF6E8B
:1063A000000EFE6E000EFD6E588BD48AD48C12A1A6
:1063B00001D0D58E12A301D0CD8012A501D0CA8400
:1063C00012A701D0B18012AF01D0F28E0BC5F8FF39
:1063D0000CC5F7FF0DC5F6FF0AC5E0FF09C5FAFFBA
:1063E00008C5FBFF02C5EAFF03C5E9FF04C5E2FFDC
:1063F00005C5E1FF06C5DAFF07C5D9FF01C5D8FF0E
:1064000000C5E8FFE1000600060058AF06D0710E97
:10641000F76EC80EF66E0BEC31F05851130B130AE1
:1064200007E0FC2A000EFF6E000EFE6E000EFD6EF1
:10643000588BD49AD48C12A101D0D58E12A301D03E
:10644000CD8012A501D0CA8412A701D0B18012AFAD
:1064500001D0F28E0BC5F8FF0CC5F7FF0DC5F6FF96
:106460000AC5E0FF09C5FAFF08C5FBFF02C5EAFF40
:1064700003C5E9FF04C5E2FF05C5E1FF06C5DAFF74
:1064800007C5D9FF01C5D8FF00C5E8FFE1009EAAF6
:1064900003D0AE509EBAFDD705EE19F00C0E166F64
:1064A000186BB1EC32F0EF6E59A105D0C0EC32F0B0
:1064B000185301E02CD0EF50EFEC32F0185303E00A
:1064C000598325D001D05993EF500D0A04E1000EF5
:1064D000EF6E4FD81CD0EF50080A0FE1190EE918E3
:1064E0000BE0080E12EC31F0200E12EC31F0080E29
:1064F00012EC31F0ED52162B08D0EE5012EC31F0C8
:10650000160703E1000EEF6E34D81653CAE11200ED
:10651000186B310A03E10A0E186F04D0030A02E176
:10652000140E186FB1EC32F0185310E00F0B18274F
:106530000A0E185F730EF76E440EF66E1851D8905F
:10654000F62601E3F72A0800F5CF18F5B1EC32F092
:106550001200E86A200E156FE806FEE11507FCE15F
:106560001200ABA202D0AB98AB889EAAFED7AE5069
:1065700012000D0E12EC31F00A0E12EC31F0120086
:106580002009136F680A02E1010E186F1351740A93
:1065900002E1020E186F13516C0A02E1030E186F2C
:1065A0001351640A02E1040E186F1351620A02E1EA
:1065B000050E186F1351770A02E1060E186F13517A
:1065C000720A02E1070E186F1351730A02E1080EF6
:1065D000186F13516D0A02E1090E186F12001B0AA1
:1065E0000AE1B1EC32F0EF6E5B0A05E1B1EC32F09A
:1065F000EF6E88EC32F01200185302E002EC33F038
:10660000196B1200FB6A660EFA6ED8901837D89094
:106610001837200ED890182501E3FA2A1851F926C8
:10662000000000002AEF33F031EF33F035EF33F0A4
:1066300040EF33F04BEF33F04EEF33F055EF33F0E4
:106640005BEF33F061EF33F064EF33F06BEF33F077
:1066500072EF33F0700EF76EBC0EF66E0BEC31F08D
:106660001200589D589BFF001200588D92D8A2D856
:106670005985280E146FA9EC32F01407FCE1FF00D5
:10668000D6EC36F0710EF76E100EF66E0BEC31F0A4
:106690001DEC37F0120008EC35F01200720EF76EA8
:1066A000720EF66EB8DD62DA120080EC31F039B9A4
:1066B00001D03981120080EC31F039B901D0398331
:1066C0001200E1EC37F01200730EF76EF20EF66E68
:1066D0000BEC31F01200730EF76EFA0EF66E0BEC47
:1066E00031F01200740EF76E020EF66E0BEC31F004
:1066F0007BEC33F0120047EC32F0050EEA6E190E17
:10670000E96E740EF76EB60EF66E0BEC31F0000EFD
:10671000F86E21EC38F037C5F7FF000EF66EFF0E6D
:10672000156F100E166F100E161911E1F850B7EC18
:1067300037F0200E12EC31F0F750B7EC37F0F638A6
:1067400010EC38F012EC31F0200E12EC31F00900B0
:10675000F6A003D0F5CF14F506D0F550B7EC37F01E
:106760001451B7EC37F0F6B003D0200E12EC31F034
:106770001607000E161908E10D0E12EC31F00A0E84
:1067800012EC31F0100E166F1507CDE1B9EC32F0B6
:106790001200000EF86EF76EF66E21EE80F029D929
:1067A000400EF626D8B0F72ADD52D952F8E1DA5277
:1067B000F6E11200396BBDEC30F0710EF76E960EFB
:1067C000F66E0BEC31F0B1EC32F03A0AD8A4FBD7FC
:1067D000326B17EC34F01F0B316FD890313317EC5C
:1067E00034F0336F17EC34F0346F17EC34F0356F4E
:1067F000010AD8B40BD03551020AD8B409D029EC1B
:1068000034F039BF13D039BD11D0DDD717EC34F0D7
:1068100080EC31F039B90AD0710EF76ED60EF66EF3
:106820000BEC31F0B1EC32F0CBEC34F01200B1EC07
:1068300032F0BF0FD8A0070F0A0F376F373BB1EC0C
:1068400032F0BF0FD8A0070F0A0F37133751322786
:10685000120005EE19F031C516F517EC34F0EE6EA6
:1068600017EC34F0EE6E162FF8D717EC34F03253E5
:10687000D8B402D0398D15D03551040AD8B407D018
:106880003551D8A40ED075D839AF0FD80AD01A51C7
:10689000300AD8A406D0B1EC32F03A0AD8A4FBD71B
:1068A00000D02E0E12EC31F01200000EF86E33C53F
:1068B000F7FFF80E3415F66E050EEA6E290EE96E36
:1068C000040E166FEFEC34F0070E3415146F290E1A
:1068D0001425E96E050EEA6E050EE26E190EE16EE4
:1068E000D890143331C516F5E6CFEEFFE6CFEEFFB4
:1068F000142B1607D8B404D01451040AD8A4F4D722
:10690000000EF86E33C5F7FFF80E3415F66E050E5F
:10691000EA6E290EE96EDDEC34F01653D8B4C1D717
:106920000900050EEA6E290EE96E16C514F5040E6F
:10693000166FEFEC34F014C516F5050EEA6E290E4D
:10694000E96EE6CFEEFFE6CFEEFF162FA1EF34F0B3
:10695000050EEA6E290EE96EF86A33C5F7FFF80EE8
:106960003415F66E080EF626D8B0F72ADDEC34F0B2
:10697000120033C55EF534C55FF531C560F5399F4A
:10698000600E335D07E605E1000E345D01E6398FE8
:1069900001D0398F1200740EF76E960EF66E0BEC66
:1069A00031F05E51B7EC37F0D8906035FE0F5F25BF
:1069B000B7EC37F0B9EC32F01200040E146F0A0095
:1069C000EECFF5FF0F00EECFF5FF0F00142FE0EF35
:1069D00034F0A68EA684FFEC34F0A69412000900D1
:1069E000F5CFEEFF0900F5CFEEFF162FEFEF34F0F5
:1069F0001200A68EA684A688FFEC34F01200D4AE56
:106A000006D0550EA76EAA0EA76EA6820000120031
:106A1000730EF76E8E0EF66E0BEC31F0730EF76E92
:106A2000540EF66E0BEC31F047EC32F005EE19F037
:106A300059B348D0EF5244E0EE52EF521EE1ED520E
:106A4000EF502009720A0AE16CEC35F0730EF76E14
:106A5000720EF66E0BEC31F03ED00ED0EF502009E6
:106A6000640A04E18EEC35F036D006D0740EF76E71
:106A7000680EF66E0BEC31F022D0ED52040E156F5D
:106A80005A8D5AAD03D0EE50B9EC36F01507F9E146
:106A90005AAD0FD0EF5206E177EC35F08EEC35F0C1
:106AA0001AD006D0740EF76E680EF66E0BEC31F04D
:106AB00006D0740EF76E680EF66E0BEC31F001D056
:106AC0000AD008D0B9EC32F0740EF76E680EF66E8C
:106AD0000BEC31F0A3D71200588D588FD4880F0ECD
:106AE000B912FF0EB86EFF0EB76ED4981200588D13
:106AF000589F05EE19F01FEEB8F0D488F00EB916C5
:106B0000020E156F21EC38F037C5E5FFEE50150782
:106B1000F9E1D890B832B732D4981200D4880F0E69
:106B2000B9140F0A1BE0730EF76E600EF66E0BECD5
:106B300031F0300E12EC31F0780E12EC31F0D890CA
:106B4000B736B836B850B7EC37F0B750B7EC37F0C7
:106B5000D890B832B732B9EC32F006D0730EF76E77
:106B6000720EF66E0BEC31F0D4981200730EF76EC5
:106B7000000EF66E0BEC31F047EC32F059B315D045
:106B800005EE19F0EF520FE022EC36F05ABF04D0B8
:106B9000DFEC35F013D006D0740EF76E680EF66E8B
:106BA0000BEC31F001D00AD008D0B9EC32F0740E01
:106BB000F76E680EF66E0BEC31F0D8D712000A0EA5
:106BC000156F15EE3AF0E7AE07D05DC5E6FF5CC580
:106BD000E6FF5BC5E7FF35D0E4505C1925E1E450E2
:106BE0005B1921E15D531AE1E552E552E2CFEAFF7C
:106BF000E1CFE9FFEE52EE52EE52150702E1E78EC9
:106C00000CD0EFBE07D0EECFE6FFEECFE6FFEECF23
:106C1000E6FF02D0E78E01D0F0D704D0E552E5526E
:106C20005DC5E7FF0ED001D0E652150708E1740EEE
:106C3000F76E7E0EF66E0BEC31F003D001D0E6520B
:106C4000C2D712005A6B5B6B5C6B5D6B05EE19F083
:106C5000030E156F5A8D5B390F0B5C6F5B39F00BB0
:106C60005B6FEF502AEC38F05B135AAD03D0EE5057
:106C7000B9EC36F01507EFE15AAD07D0060E5C5DB2
:106C800004E65C510F0A01E05A9D5AAD54D0EF5210
:106C900001E150D0EF502009200A47E0EF502009D1
:106CA000610A09E1300E5D1504E1300E300B5D1311
:106CB00001D05A8F3AD0EF502009620A12E1300E0B
:106CC0005D150DE15D510F0B08E15DBD04D0300E87
:106CD000200B5D1301D05A8F01D05A8F01D05A8FEB
:106CE00024D0EF502009680A09E1300E5D1504E157
:106CF000300E100B5D1301D05A8F17D0EF502009C2
:106D00002D0A0CE15DBD08D05D51300B200A02E078
:106D10005D8D01D05A8F01D05A8F07D05D510F0B76
:106D200003E1A5EC36F001D05A8F5AAF01D002D062
:106D3000EC52ADE101D05A8F5ABF06D05D510F0B16
:106D400003E15DAD01D05A8F1200EF5020093108E8
:106D50000EE7090F0AE65D51300B200A02E15A8F57
:106D600003D0EF500F0B5D1301D05A8F01D05A8F13
:106D700012005A9D2009146F2F080AE70A0F02E635
:106D80005A8D06D01451600803E7060F01E65A8DAC
:106D90001200050EE26E3A0EE16E0A0E146F800EBE
:106DA000E66EE66AE66A1407FAE11200720EF76E02
:106DB000E20EF66E0BEC31F001D8120015EE3AF04F
:106DC0000A0E156FE7AE02D035D02ED0E7CF5DF5B5
:106DD000E45010EC38F012EC31F0E450B7EC37F03E
:106DE0005DAD02D02D0E01D0200E12EC31F05D51C0
:106DF000300B300A08E15D510F0BFB0F02E6020F6A
:106E000001D0010E0FD05D51300B200A02E1050EBA
:106E100009D05D510F0BFD0F02E6010F01D0000EEE
:106E2000E846010FDAEC37F0150702E103D001D094
:106E3000E652C8D7B9EC32F012000E5198D80F5173
:106E400096D8010EB7D8005192D8010EB3D801A53B
:106E500002D0310E01D0300E12EC31F0200E12ECC7
:106E600031F001A102D0310E01D0300E12EC31F020
:106E7000200E12EC31F001A902D0310E01D0300EFB
:106E800012EC31F0010E96D802516DD803516FD833
:106E9000020E90D8045167D8055169D8020E8AD8DD
:106EA000065161D8075163D8020E84D85BEC37F0E5
:106EB000B9EC32F0120015EE3AF00A0E156FE7AE9B
:106EC00002D02DD026D0E7CF5DF5E4CFEAFFE4CFA6
:106ED000E9FF5D510F0B01E15D2B050E146F5DBDE8
:106EE00008D090EC37F0EE525D075D510F0BF9E1E1
:106EF0000DD05D510F0BFF0FE92601E3EA2A90EC5C
:106F000037F0ED525D075D510F0BF9E11451DAECEA
:106F100037F0150702E103D001D0E652D0D71200B6
:106F20005D51300B300A0AE1EF50CEEC37F012EC35
:106F300031F01451FF0F01E0140714D05D51300BF4
:106F4000200A06E1EF50C1EC37F0010E146F0AD0B1
:106F5000EF50B7EC37F01451050A02E1030E01D0EF
:106F6000010E146F12005CD812EC31F01200136F96
:106F7000133956D812EC31F0135152D812EC31F0CB
:106F80001200136F080E166F133702E3310E01D093
:106F9000300E12EC31F01607F7E11200136F810F7B
:106FA00002E32A0E06D01351E00F02E22A0E01D0AE
:106FB00013511200136F200E12EC31F01307FCE195
:106FC0001200710EF76E140EF66E0BEC31F047ECFA
:106FD00032F005EE19F0EF503DD8386FEC5021EC4F
:106FE00038F037C536F5EC5003E1FBEC37F002D052
:106FF00017EC38F01200710EF76E720EF66E0BEC95
:1070000031F038C5E2FF36C5E1FFE73809D812ECA8
:1070100031F0E75005D812EC31F0B9EC32F0120043
:107020000F0BF60F02E23A0F01D0410F120038C5E4
:10703000E2FF36C5E1FFEC5021EC38F037C5E7FF41
:107040001200EF5007D8376F373BEC5003D8371397
:107050003751120020099F0F02E30A0F01D0310FB0
:107060001200FC060D0E12EC31F00A0E12EC31F09B
:10707000FC50B7EC37F03A0E12EC31F0FE50B7ECA2
:1070800037F0FD50B7EC37F00D0E12EC31F00A0E70
:1070900012EC31F0FC2A12000D0A09090951776936
:1070A0006B42756720666F72205049433138463411
:1070B00035322076312E322E330D0A000D0A46313C
:1070C0000946320946330946340946350946360928
:1070D00046370946380946390D0A48656C70097209
:1070E00065736554094C6F616409446973706C6120
:1070F0007909427265616B09576174636809527559
:107100006E0953746570094D6F646966790D0A00E4
:1071100051423E00446973706C61792F4D6F646910
:10712000667920636F6E74656E7473206F6620528B
:10713000414D206F722072656769737465722061BA
:107140006464726573733A200D0A3C6161613E208C
:10715000746F20446973706C6179202C3C616161AB
:107160002078783E20746F204D6F646966790D0A2F
:107170000000436F6E74656E74732028486578292B
:107180003A200000457261736520436F6D706C6535
:1071900074652E2E2E00557365722070726F6772A3
:1071A000616D206D656D6F727920657261736564C4
:1071B000202D2053656E64204845582066696C6513
:1071C000206E6F770D0A000052756E6E696E672E25
:1071D0002E2E0D0A00000D0A446F776E6C6F6164ED
:1071E000207375636365737366756C0D0A000D0A11
:1071F0005472616E736D6974204572726F72202DC6
:1072000020436865636B73756D0D0A000D0A577234
:107210006974696E67206F7574736964652055734E
:107220006572204164647265737320537061636595
:107230000D0A00000D0A4E6F207573657220636F92
:10724000646520726573657420766563746F72205F
:107250006973206C6F616465640D0A004E6F205580
:1072600073657220436F6465204C6F616465640DC3
:107270000A00456E746572207761746368207661D8
:10728000726961626C652E204578616D706C657302
:107290003A207C20303132207C2030313220622074
:1072A0007C2030313220612038207C203031322067
:1072B00032207C203031322032202D207C0D0A00FB
:1072C0004D75737420626520616E20416363657340
:1072D000732042616E6B20616464726573730D0A82
:1072E000000020504320205720205A2043204E20C9
:1072F00046535230204653523120465352322000DA
:107300002046363E000009095177696B42756720B7
:107310004175746F7374617274696E67205573651B
:107320007220436F64650D0A00000909507265738D
:107330007320616E79206B657920746F2061626FB4
:107340007274200000010203040500060708090A00
:10735000000B0C002046353E0000202042503E002D
:1073600020202020427265616B706F696E74203D31
:107370002000202020204E6F20627265616B706FAC
:10738000696E74206973207365740D0A00003C6196
:107390006161613E20746F20736574206272656163
:1073A0006B706F696E742C2027522720746F2072C7
:1073B000656D6F766520627265616B706F696E7462
:1073C0002C2027442720746F20646973706C6179C6
:1073D00020627265616B706F696E740D0A00526590
:1073E00073657420436F6D706C6574652E200A0D93
:1073F0000000463130200D0A0000463131200D0AD0
:1074000000004631323A456E7465722048696768FB
:107410002041646472657373283220686578206443
:107420006967697473293E0042726F776E2D6F75BC
:107430007420526573657420446574656374656473
:107440000A0D0000537461636B204F766572666CA1
:107450006F770A0D0000537461636B20556E64658D
:1074600072666C6F770A0D002046363E496E766173
:107470006C696420436F6D6D616E640A0D00204677
:10748000363E576174636820417272617920467597
:107490006C6C0A0D0000486967686573742041646C
:1074A00064726573732050726F6772616D6D65648D
:1074B0003A20307800002020202020202030203169
:1074C0002020322033202034203520203620372041
:1074D00020382039202041204220204320442020F1
:0674E0004520460D0A00E4
:020000040030CA
:0E000000FFFAFCFEFFFF7BFFFFFFFFFFFFFF8D
:00000001FF
